:1003C300110E3031323334353637383941424344F4
:0303D3004546009C
:10000300E4FFFE12037F1203D7D2017590FFD2974C
:09001300D295C29412035580FB42
:04037B007F2C7E0154
:10037F00E4FDFCD3ED9FEC9E5015E4FBFA0BBB00A4
:0F038F00010AEB646F4A70F50DBD00010C80E4AC
:01039E00223C
:10035500300022C200E50A24FE600F14600F14600D
:100365001124037010AF0B0201E10202BAAF0B02B8
:0603750001331200B22268
:0201E1008F216C
:1001E300120287E509646970383001FDC20175990F
:1001F3000112037BE4F522D3E5216480F8E5226450
:1002030080985009AF22120231052280EAC294D2AB
:10021300973001FD7F037E0012037FC201759903AE
:0D022300223001FDC201759902C294D297EC
:0102300022AB
:0E0279007FF47E0112037FC294D29712037F9E
:10028700C297D294D2947F327E001203327F5312E8
:100297000337E4FF120337E4FFE52325E030960533
:1002A70004F5238002F523D297C2970FBF08EA858A
:0202B700230919
:0102B9002222
:1002BA00120287E5096469702612032E7F801203F1
:1002CA0037E4FF120337E4FF1203377FF47E01128B
:1002DA00037FC294D2973001FDC201759901223081
:0C02EA0001FDC201759902C294D2972256
:020133008F211A
:10013500D2021202BA12037B120287E509646970C2
:100145003912037B3001FDC201759930E4F522AF08
:1001550021EF3395E0FED3E5229FEE6480F87480AD
:10016500985009AF2212018C052280E3C294D297E0
:100175007F647E0012037FC202223001FDC2017539
:060185009902C294D2971A
:01018B002251
:02018C008F23BF
:10018E007F50120337AF23120337E4F524F52530E1
:10019E0003FDC203E525F4452470047F0180027F30
:1001AE0000E523B50B047E0180027E00EE5F700831
:1001BE003001FDC201759930AF0D120337E4FFFE19
:1001CE0012037F0525E52570020524C3E52494015D
:0201DE0040BD22
:0101E00022FC
:020231008F2319
:100233007F30120337AF23120337E4F525F526E4A5
:10024300FFE52425E030960504F5248002F524D249
:1002530097C2970FBF08EA7F017E0012037FAF2486
:1002630012039FE4F5240526E52670020525C3E560
:0502730025940140CAC2
:010278002263
:1000B200120287E5096469706B12032E7FE0120356
:1000C20037E4FF120337E4FF1203371202797FACE1
:1000D2001203377FE1120337E4FF120337E4FF1202
:1000E20003371202797FAC1203377FE2120337E43F
:1000F200FF120337E4FF1203371202797FAC1203B7
:10010200377FE3120337E4FF120337E4FF120337AA
:100112007FF47E0112037FC294D2973001FDC201A7
:10012200759901223001FDC201759902C294D297DC
:0101320022AA
:09032E007FF47E0112037F7FAC15
:10033700E4FEEF30E704D2958002C295D297C297C8
:0E034700EF25E0FF0EBE08EAE4FFFE02037F92
:030023000202F6E0
:0902F600C0E0C0D075D000C000CA
:1002FF00309821C29830020785990DD20380197466
:10030F000A2508F8A6990508E508B4020BD200756E
:08031F0008008004C299D2011C
:07032700D000D0D0D0E0327D
:10039F003001FDC201EF7804A2E713D8FB540F24FC
:1003AF000EF8E6F5993001FDC201EF540F240EF857
:0403BF00E6F59922A4
:1003D700758920438780758DFDD28E75985075A8D5
:0203E700902262
:03000000020026D5
:0C002600787FE4F6D8FD75812602006D9D
:10003200020003E493A3F8E493A34003F68001F2E1
:1000420008DFF48029E493A3F85407240CC8C333CF
:10005200C4540F4420C8834004F456800146F6DF9E
:10006200E4800B01020408102040809003C3E47E68
:10007200019360BCA3FF543F30E509541FFEE49393
:10008200A360010ECF54C025E060A840B8E493A35A
:10009200FAE493A3F8E493A3C8C582C8CAC583CA85
:1000A200F0A3C8C582C8CAC583CADFE9DEE780BE3D
:0103D6000026
:00000001FF
